:020000000528D1
:08000800DE2817203E2007301E
:10001000A100D520A10B0928972068205320073084
:10002000A100D520A10B112897206820062883164F
:1000300007309F008501860104308700F03088007A
:100040008901F930920004308C0001308D00243099
:1000500098001930990083124D30920000309000C2
:10006000053097000A309D008501860187018801CF
:10007000890180309800C0308B000800E8309B0078
:1000800003309C008E018F0195019601860102309C
:10009000A700061410148C3084000011D9208C3075
:1000A000840000150800E8309B0003309C008E019E
:1000B0008F019501960186012030A70006161014C5
:1000C0008C3084000011D9208C3084000015080089
:1000D0000C1E68282B0899000C1E6C282A08990011
:1000E0000C1E70282A0899000C1E742829089900F3
:1000F0000C1E7828290899000C1E7C2828089900D5
:100100000C1E8028280899000C1E84280D309900A8
:100110000C1E88280D3099000C1E8C280A3099007E
:100120000C1E90280A3099000C1E94280800220802
:10013000A1000F30A1050A302102031CA3282103CE
:100140000739403EA5282108303EA8002208A1001A
:10015000A10E0F30A1050A302102031CB328210390
:100160000739403EB5282108303EA9002308A100E8
:100170000F30A1050A302102031CC22821030739D0
:10018000403EC4282108303EAA00230EA1000F30B3
:10019000A1050A302102031CD12821030739403E62
:1001A000D3282108303EAB0008008C1CD5288C10C9
:1001B00008002830A100A10BDB280800A400030ED2
:1001C000A5000C19EA280D18F328250E8300A40EAB
:1001D000240E09000C1110101508A2001608A30027
:0E01E000D5208601E1280D1027088606E128AB
:02400E00B13FC0
:00000001FF
